:1000000028C041C03FC05AC03DC01DC17BC03AC0DE
:1000100039C038C037C036C035C034C033C032C034
:1000200031C030C02FC0CBC1D4C1D7C1D8C1D9C114
:10003000DAC1DBC1DCC1DDC1DEC1DFC1E2C12AC280
:100040002EC237C240C249C252C25BC264C26DC234
:1000500076C211241FBECFEDCDBF10E0A0E6B0E008
:10006000E6E2F7E003C0C89531960D92A036B107DD
:10007000D1F710E0A0E6B0E001C01D92A037B107B3
:10008000E1F7AEC2BDCF1F920F920FB60F921124AF
:100090008F931DBC1CBC88ED82BF88B7826888BF67
:1000A00089B78A6089BF809167008160809367000B
:1000B0008F910F900FBE0F901F9018951F920F9267
:1000C0000FB60F9211242F933F934F938F939F93CB
:1000D00089B7877F89BF24B535B5932F822F845880
:1000E0009340815B944020F430936500209364003A
:1000F0009F918F914F913F912F910F900FBE0F9035
:100100001F9018951F920F920FB60F9211242F93E4
:100110003F938F939F938091670080FF10C08091E1
:1001200067008E7F80936700809167008260809374
:100130006700809167008860809367007BC0809132
:10014000670083FF3BC08091680085FD0CC0209153
:1001500062003091630080916E0090916F00821771
:10016000930780F014C08091680085FF18C020912B
:1001700062003091630080916E0090916F002817AB
:10018000390728F4809160009091610004C080914B
:1001900062009091630090936A0080936900C19A15
:1001A00089B7806889BF8091690090916A008095C5
:1001B00090959DBD8CBD8BEE82BF3CC08091670049
:1001C00084FF38C08091680085FD0CC020916200DA
:1001D0003091630080916E0090916F00281739076D
:1001E00080F014C08091680085FF18C020916200E3
:1001F0003091630080916E0090916F008217930799
:1002000028F4809160009091610004C080916200A8
:100210009091630090936A0080936900C09A8091E6
:10022000690090916A00809590959DBD8CBD89B7BD
:100230008D7F89BF9F918F913F912F910F900FBE1E
:100240000F901F9018951F920F920FB60F921124C6
:100250008F939F938091670083FF0CC0C19880911A
:100260006700877F8093670080916700806180933B
:10027000670056C08091670084FF0AC0C0988091D3
:1002800067008F7E8093670089B78F7789BF48C0EA
:100290008091670085FF25C0859918C080916D0009
:1002A000982F8F5F80936D009630C0F084990CC0BA
:1002B000949A80916C008F5F80936C009927880FCF
:1002C000991F80936B000AC0949808C080916700C2
:1002D0008F7D80936700949810926D008BED9BE06A
:1002E00012C08091670086FF1BC080916B00815017
:1002F00080936B008F3F51F0849902C0949A01C0A3
:1003000094988DEE95E89DBD8CBD0AC080916700E4
:100310008F7B80936700949810926B0010926C0012
:100320009F918F910F900FBE0F901F90189585E0B1
:1003300083BF82E08EBD83E085BF8BB780648BBFB7
:10034000789483E087BB80E181BB959A0895A1E012
:10035000B0E0D3D1F0936F00E0936E00A0E0B0E086
:10036000C4D1802D80936800AFE7B0E0BED1802D6E
:1003700099278093660081BF0895A1E0B0E0E199DC
:10038000FECF80916E0090916F00082E192EC6D17D
:10039000A0E0B0E0E199FECF80916800082EB2D1D4
:1003A000089580916C009927AA27BB27F92FE82F81
:1003B0003197EC30F10548F5ED5EFF4F09948091DF
:1003C00064009091650090936F0080936E0081E0CF
:1003D00001C082E080936800089583E0FBCF84E051
:1003E000F9CF85E0F7CF86E0F5CF87E0F3CF88E05F
:1003F000F1CF89E0EFCF8AE0EDCF80916800806196
:10040000E9CF809168008062E5CF809168008F70AD
:10041000E1CF209164003091650080916E00909151
:100420006F00281B390B37FF04C080916700846080
:1004300003C0809167008B7F809367008091680084
:1004400084FF0DC08091670082FF04C08091670027
:100450008B7F03C080916700846080936700932F37
:10046000822F37FF03C0909581959F4F9093630033
:1004700080936200809168008F709927AA27BB271C
:10048000F92FE82F3197EA30F10508F068C0E15EF6
:10049000FF4F099480916200909163005CC080914D
:1004A00062009091630064E670E0F7D06EE670E061
:1004B0004FC0809162009091630064E670E0EDD0DF
:1004C00068E770E045C0809162009091630064E647
:1004D00070E0E3D062E870E03BC0809162009091F0
:1004E000630064E670E0D9D06CE870E031C08091C0
:1004F00062009091630064E670E0CFD066E970E03E
:1005000027C0809162009091630064E670E0C5D0DE
:1005100060EA70E01DC0809162009091630064E623
:1005200070E0BBD06AEA70E013C0809162009091E5
:10053000630064E670E0B1D064EB70E009C08091C4
:1005400062009091630064E670E0A7D06EEB70E00B
:10055000B6D0972F862F9093610080936000809192
:10056000670082FF0DC08091620090916300880F48
:10057000991F2091620030916300281B390B04C041
:10058000209162003091630080916E0090916F0025
:10059000280F391F30936300209362008091670019
:1005A00082FF0DC08091600090916100880F991FBB
:1005B0002091600030916100281B390B04C020910C
:1005C00060003091610080916E0090916F00280F63
:1005D000391F30936100209360008FEF82BF089530
:1005E000CFEDD0E0DEBFCDBF88E190E02BE00FB6CD
:1005F000F894A89581BD0FBE21BDA9DE98DEA8950F
:10060000859940C088B38C7F88BB88E10FB6F89489
:1006100081BD11BC0FBE8BB78F7B8BBF89B7857F28
:1006200089BF83E08EBD88B7826888BF8BED9BE071
:100630009DBD8CBD89B7806889BF80E280936700CB
:100640008091670085FDFCCF89B78F7789BF809146
:100650006C00882309F4C8CFA4DE8FDE88B78268D7
:1006600088BF8DEE95E89DBD8CBD8091670080644C
:100670008093670089B7806889BF8091670086FD95
:10068000FCCFB2CF8091670081FFB9CF8091670026
:100690008D7F80936700BDDEB2CF5527002480FF99
:1006A00002C0060E571F660F771F6115710521F0F6
:1006B00096958795009799F7952F802D0895AA1BF9
:1006C000BB1B51E107C0AA1FBB1FA617B70710F03D
:1006D000A61BB70B881F991F5A95A9F7809590956F
:1006E000682F792F8A2F9B2F0895E199FECFBFBBEA
:1006F000AEBBE09A11960DB20895F7DFE02DF5DF5D
:10070000F02D0895E199FECFBFBBAEBB0DBA119697
:100710000FB6F894E29AE19A0FBE0895F3DF012C28
:06072000F1DF1124089531
:00000001FF
